:100000000C947F020C94B7020C94B7020C94B702C4
:100010000C94B7020C94B7020C94B7020C94B7027C
:100020000C94B7020C94B7020C942C270C94FE2766
:100030000C940B220C94B7020C94B7020C94B702E8
:100040000C94B7020C94B7020C94B7020C94B7024C
:100050000C94B7020C9493220C94B7020C94B70240
:100060000C94B7020C94B7020C94B7020C94B7022C
:100070000C94B7020C94B7020C94B7020C94B7021C
:100080000C94B7020C94B7020C94B7020C94B7020C
:100090000C94B7020C94B7020C94B7020C94B702FC
:1000A0000C94B7020C94B7020C94B702FF04FF043F
:1000B0002B052B059305B105C906C906BC055506D8
:1000C000660666066B2892288A2992288A29DE28E5
:1000D00001298A2958296729165C1E001F00200063
:1000E00021002200230024002500260027002D00E7
:1000F0002E0031002A0049002B00000014001A00D5
:100100000800150017001C0018000C001200130056
:100110002F00300031004C003900000004001600B0
:10012000070009000A000B000D000E000F0033004D
:100130003400280000004B00E10064001D001B009B
:1001400006001900050011001000360037003800C5
:100150000000E50052004E00E000E3000000E20075
:100160002C0000002C0000002C000000E600E7003E
:10017000E400500051004F0000047F3F1F64321420
:10018000643214783C1E1E140A05222325262829D1
:100190002A2C2D2F3032333536383A3B3D3E404203
:1001A000434547494A4C4E5051535557595A5C5E46
:1001B0006062646668696B6D6F71737577797B7D5A
:1001C0007F81838587898A8C8E90929496989A9C59
:1001D0009E9FA1A3A5A7A8AAACAEAFB1B3B4B6B871
:1001E000B9BBBCBEBFC1C2C3C5C6C7C9CACBCCCDD3
:1001F000CED0D1D2D2D3D4D5D6D7D7D8D9D9DADAAE
:10020000DBDBDBDCDCDCDCDCDDDDDDDDDCDCDCDC2D
:10021000DCDBDBDBDADAD9D9D8D7D7D6D5D4D3D261
:10022000D2D1D0CECDCCCBCAC9C7C6C5C3C2C1BF3F
:10023000BEBCBBB9B8B6B4B3B1AFAEACAAA8A7A5A3
:10024000A3A19F9E9C9A98969492908E8C8A89875F
:100250008583817F7D7B79777573716F6D6B69683D
:10026000666462605E5C5A5957555351504E4C4A11
:100270004947454342403E3D3B3A383635333230BC
:100280002F2D2C2A292826252322FFAA7F5540001E
:100290000101010101010101010202020202020247
:1002A000020203030303030303030404040404041A
:1002B00004050505050506060606060707070707E0
:1002C00008080808090909090A0A0A0B0B0B0C0C93
:1002D0000C0D0D0D0E0E0E0F0F0F1010111111122F
:1002E0001213131414151516161717181819191AAE
:1002F0001A1B1B1C1D1D1E1E1F2020212222232411
:1003000024252626272829292A2B2C2D2D2E2F304F
:10031000313232333435363738393A3B3C3D3E3F63
:10032000404142434445464748494A4C4D4E4F5050
:10033000515354555658595A5B5D5E5F616264650E
:100340006668696B6C6D6F7072737577787A7B7D98
:100350007E8082838587888A8C8E8F9193959698EC
:100360009A9C9EA0A2A3A5A7A9ABADAFB1B3B5B708
:10037000BABCBEC0C2C4C6C9CBCDCFD1D4D6D8DBDF
:10038000DDDFE2E4E7E9EBEEF0F3F5F8FAFDFF1C60
:10039000034B004500590043004C00410043004B13
:1003A00000360035002D00560031000000080364BF
:1003B000006F00750000000403090409023B0002FD
:1003C0000100A0FA09040000010301010009211144
:1003D0000100012240000705810308000109040112
:1003E00000010300000009211101000122B60007ED
:1003F0000582032000011201000200000008EDFE4A
:10040000606002000102000105010902A1018502EC
:100410000901A10005091901290815002501950800
:10042000750181020501093009311581257F950289
:100430007508810609381581257F950175088106A3
:10044000050C0A38021581257F950175088106C0C3
:10045000C005010980A101850319012AB700150112
:1004600026B700950175108100C0050C0901A10196
:10047000850419012AA002150126A0029501751014
:100480008100C005010906A1018506050719E029BB
:10049000E715002501950875018102050719002956
:1004A000EF1500250195F075018102050819012954
:1004B00005950575019102950175039101C005012E
:1004C0000906A101050719E029E71500250195088E
:1004D000750181029501750881010507190029FF41
:1004E000150026FF009506750881000508190129E9
:1004F00005950575019102950175039101C01124BF
:100500001FBECFEFDAE0DEBFCDBF04B603FE18C0DA
:1005100080914B0390914C03A0914D03B0914E03F9
:100520008730904BA740B04B59F410924B03109278
:100530004C0310924D0310924E03E0E0F8E309954E
:1005400011E0A0E0B1E0EAE9F5E502C005900D9206
:10055000A83CB107D9F723E0A8ECB1E001C01D9297
:10056000AB34B207E1F70E94C0120C94CB2A0C9472
:10057000000081E0089581E008950C94BB02089585
:100580000C94BF021F93CF93DF9300D000D01F9233
:10059000CDB7DEB749835A836B833091CB01898114
:1005A0009A81311114C0662359F0222349F00E9428
:1005B0000609182F682F89819A810E94AF0803C00D
:1005C0000E94DA08182F69817A81812F04C00E9465
:1005D000060969817A810F900F900F900F900F900C
:1005E000DF91CF911F910C944010FC01262F408188
:1005F00051816281738184810C94C20281E00895EB
:10060000CF93DF93EC0160E00E94F502BE01DF9121
:10061000CF910C94C0020C9471110C946D1108953B
:100620000E9459070E940F032FEF84E39CE02150A2
:1006300080409040E1F700C000000C94B9220F9375
:100640001F93CF93DF938C0161E00E94F502EC01D0
:10065000B8010E94BD02882309F44BC0B801CE0145
:100660000E94441D882309F444C0B801CE010E94B1
:1006700056208823F1F1B801CE010E946A1E88231A
:10068000C1F1B801CE010E94B21F882391F1B801D7
:10069000CE010E94881B882361F1F80182818823A2
:1006A00009F1CB358DE5D807C1F050F4C115FCE553
:1006B000DF0781F0CF3DDC45A9F40E94370E19C059
:1006C000CC35EDE5DE0761F0CD35DD4559F40E940E
:1006D000800D08C00E9410030CC00E94890D02C04A
:1006E0000E948C0DC801DF91CF911F910F910C9446
:1006F000B90280E0DF91CF911F910F9108950E9480
:10070000ED2180E00E94791D0C94AA030E94681CD0
:100710000E94AD030C94F32108950C948C0381E0A6
:100720000895CF93C82F0E948F03882329F0C1FD1D
:1007300002C02A9A01C02A98CF910895229A2A9A33
:100740000895CF93C82F0E948D038C2F0E94910390
:10075000CF91089580E00C94A1030E94B2200C94E4
:10076000A1030E94B2209091CA01891721F08093C1
:10077000CA010C94A1030895CF93DF93CDB7DEB7E0
:100780002B970FB6F894DEBF0FBECDBF4F835887AF
:1007900069877A878B8761110E94CC0C9E012F5F3D
:1007A0003F4F86E0F90111928A95E9F785E0FE0155
:1007B0003796D90101900D928A95E1F789819A8146
:1007C0004C815D81452B31F09F3F31F491E08F3FAB
:1007D00019F403C091E001C090E090FF09C0498185
:1007E0005A816B817C818D819E810E94ED0B05C0B9
:1007F000C9010E94FE028111F2CF2B960FB6F89428
:10080000DEBF0FBECDBFDF91CF910895FC01808187
:1008100091810E9448090895CF93882309F450C01C
:10082000C82F8CEF8C0F813AD0F46C2F809102018D
:10083000909103010E942821882349F06C2F809118
:100840000201909103010E94B3210E94EE0C6C2FD3
:1008500080910201909103010E94A8210CC080E2C6
:100860008C0F883058F4C77081E001C0880FCA959A
:10087000EAF70E94AF0CCF910C94EE0CEBE5EC0F75
:10088000E33040F4F0E0E65AFE4F808190E0CF91F3
:100890000C94E620E8E5EC0FE73150F4F0E0EE0FC1
:1008A000FF1FE45DFE4F80819181CF910C94FC206D
:1008B000CD3E30F08C2F0E944513CF910C9417142D
:1008C000CF910895882389F19CEF980F913A40F4D5
:1008D000682F80910201909103010E94B3210DC005
:1008E00090E2980F983058F4877091E001C0990F0A
:1008F0008A95EAF7892F0E94B50C0C94EE0C9BE5C3
:10090000980F933020F480E090E00C94E62098E576
:10091000980F973120F480E090E00C94FC208D3EFD
:1009200020F00E94A0130C94171408951F93CF93E6
:10093000DF93182FEB010E940C04209741F08FE900
:100940009FE00197F1F700C000002197F6CF812FBB
:10095000DF91CF911F910C946204893319F060E00C
:1009600070E002C060E570E00C949604882321F0EA
:100970000E94AF0C0C94EE0C0895882321F00E9485
:10098000B50C0C94EE0C0895CF92DF92EF92FF928B
:100990000F931F93CF93DF937C01D62FC72FFC01BA
:1009A0001281058102950F700E94A50C8823B9F071
:1009B0001123A9F08C2F807F803421F080E28D0FED
:1009C000883068F08091E30282FD09C082E00E94D5
:1009D0004E0D0E94A50C91E0D82ED92601C0D12C35
:1009E000CC2EC2948FE0C8228C2D90E08C309105E3
:1009F00008F0CFC1FC01EA5AFF4F0C94262A8C2F35
:100A0000807FCF70882311F0C295C07F112399F0A9
:100A1000CC2309F4AAC180E28D0F883010F0D111E7
:100A200004C08C2F0E94AF0C03C08C2F0E94BF0CFF
:100A30000E94EE0C9AC18D2F0E946204CC2309F40F
:100A4000A8C180E28D0F883038F1DD2329F18C2F89
:100A50000E94C50C24C08C2F807FCF70803211F093
:100A6000C295C07FDD2319F0D130A1F13DC0809146
:100A7000E30282FF17C0112349F0CC2329F08C2F09
:100A80000E94AF0C0E94EE0C80E070C180E00E94DA
:100A90006204CC2309F47DC18C2F0E94B50C0E9406
:100AA000EE0C77C1112371F0002341F0013031F4D5
:100AB0000E94CF0C8C2B0E94D70C6BC10E94CF0CD4
:100AC0008C2B1DC0002319F0013009F462C10E9473
:100AD000E40C25C0112321F0063008F05AC10EC0E5
:100AE000053008F056C11BC0112361F0002331F01E
:100AF000F701858180FF39C18F7085838C2F0E941B
:100B0000B60447C1002359F0D93309F03FC1FFEFC4
:100B100007EE13E0F15000401040E1F735C18C2F93
:100B20000E94BD0436C18C2F86958695837019F07E
:100B3000813061F02EC1112321F08D2F9C2F9370F5
:100B400002C080E090E00E94E6202BC1112321F03A
:100B50008D2F9C2F937002C080E090E00E94FC20BB
:100B600020C18D2F112319F00E94451302C00E944D
:100B7000A0130E94171415C18C2F837009F047C071
:100B800011110BC12D2F229526952770220F220FB0
:100B90006D2F6F70862F90E0A0E0B0E0022E04C0B1
:100BA000880F991FAA1FBB1F0A94D2F7D4FF10C049
:100BB0004FE050E060E070E004C0440F551F661F36
:100BC000771F2A95D2F7409550956095709503C090
:100BD00040E050E0BA01C695C695C3708A019B01FA
:100BE000082B192B2A2B3B2BC901B801C23049F025
:100BF00058F4C13019F00E94C507CFC00E94B30756
:100C0000CCC00E94D707C9C00E94B107C6C011233B
:100C100019F08C2F817001C08695882309F4BDC01E
:100C20002D2F229526952770220F220F6D2F6F7082
:100C3000862F90E0A0E0B0E0022E04C0880F991F3C
:100C4000AA1FBB1F0A94D2F7D4FF10C04FE050E098
:100C500060E070E004C0440F551F661F771F2A959F
:100C6000D2F7409550956095709503C040E050E0F4
:100C7000BA01C695C695C3708A019B01082B192B32
:100C80002A2B3B2BC901B801C23049F058F4C130BE
:100C900019F00E948A0881C00E9478087EC00E94D4
:100CA0009C087BC00E94EB0778C0CF70112339F0FD
:100CB0008C2F0E9411088D2F0E94B6046EC08D2FBC
:100CC0000E94BD048C2F0E94320867C0D23F21F1E0
:100CD00028F4D03F41F0D13FC1F043C0D33F19F1D8
:100CE000D43F79F03EC0112341F0053008F051C0E7
:100CF0008C2F8F710E9457084CC0063008F049C0F5
:100D0000F7CF8091E30282FF18C0112339F08C2FB6
:100D10008F710E9411083DC01123C9F38C2F8F7170
:100D20000E94320836C0112329F08C2F8F710E9447
:100D3000FC072FC00E94F7072CC0112349F0CF7188
:100D40008C2F0E94110863E08C2F0E94330D21C06C
:100D500081E00E944E0D0230E0F082E00E944E0DD4
:100D600018C0112331F0002391F28D2F0E940C0442
:100D700010C0002399F2D93349F41FEF27EE33E076
:100D8000115020403040E1F700C000008D2F0E943C
:100D9000620488EF8C0D843020F40E94B2200E94FF
:100DA000A103DD20C9F00E94A10C80FD15C0F70150
:100DB00012820E949B0C0E941108C7010E940D071D
:100DC0000E949B0CDF91CF911F910F91FF90EF90AC
:100DD000DF90CF900C943208DF91CF911F910F914B
:100DE000FF90EF90DF90CF9008950F931F93CF93D4
:100DF000DF93EC01688179818A810E9453098C011B
:100E00000E94AE080E949F07B801CE010E94C40450
:100E1000DF91CF911F910F910895CF93DF93EC0154
:100E2000988189812B813C81232B31F08F3F31F4D4
:100E300081E09F3F19F403C081E001C080E080FDA4
:100E40001DC0CE010E941F03811110C00E94A50C7D
:100E50008823A1F08A81882389F08091E30282FDB2
:100E60000DC082E0DF91CF910C944E0DCE010E9417
:100E7000F506CE01DF91CF910C940003DF91CF9165
:100E8000089580E090E00E94E62080E090E00E94DB
:100E9000FC200E94CC0C0E94EE0C0E9448150C9481
:100EA000171480910201909103010E94BE210C94BD
:100EB00041070E94BC0C0C94510792959F7096308C
:100EC00079F010F4925001C09A50923068F4803F4B
:100ED00069F018F4883E40F409C0843F29F406C044
:100EE000883E20F0813F11F080E0089581E0089570
:100EF000FC01808191810E9448090E945D0708954C
:100F0000CF93DF9300D000D01F92CDB7DEB70F9004
:100F10000F900F900F900F90DF91CF910895CF9386
:100F2000DF9300D000D000D0CDB7DEB726960FB645
:100F3000F894DEBF0FBECDBFDF91CF910895089525
:100F400008950C94A0070C94A1070E94A307609336
:100F500002027093030280930402909305020C94A2
:100F600041070C94A5070F931F9300910202109163
:100F700003022091040230910502602B712B822B19
:100F8000932B1F910F910C94A5070F931F93009122
:100F900002021091030220910402309105026023A5
:100FA0007123822393231F910F910C94A5070F9314
:100FB0001F930091020210910302209104023091CC
:100FC000050260277127822793271F910F910C94A8
:100FD000A5070C94A0070E94E9076093FE01709397
:100FE000FF0180930002909301020C94410760E09E
:100FF00070E0CB010C94EB070F931F9341E050E09E
:1010000060E070E08A019B0104C0000F111F221FE5
:10101000331F8A95D2F7C901B8011F910F910C9423
:10102000EB070F931F9341E050E060E070E004C0D5
:10103000440F551F661F771F8A95D2F78091FE01D6
:101040009091FF01A0910002B09101028A019B01E1
:10105000082B192B2A2B3B2BC901B8011F910F918B
:101060000C94EB070F931F9341E050E060E070E0B9
:1010700004C0440F551F661F771F8A95D2F740950D
:101080005095609570958091FE019091FF01A0911F
:101090000002B09101028A019B01082319232A232F
:1010A0003B23C901B8011F910F910C94EB070F93DB
:1010B0001F9341E050E060E070E004C0440F551F12
:1010C000661F771F8A95D2F78091FE019091FF01EC
:1010D000A0910002B09101028A019B010827192703
:1010E0002A273B27C901B8011F910F910C94EB07E8
:1010F0000F931F930091FE011091FF0120910002B8
:1011000030910102602B712B822B932B1F910F9139
:101110000C94EB070F931F930091FE011091FF01B8
:1011200020910002309101026023712382239323D6
:101130001F910F910C94EB070F931F930091FE01E9
:101140001091FF0120910002309101026027712768
:10115000822793271F910F910C94EB07089520E1AC
:10116000929F800D1124E82FE695E695E69587700D
:1011700051E001C0550F8A95EAF785E0E89FF0013C
:101180001124E453FE4F20E030E070E04081CB01B9
:10119000022E02C0969587950A94E2F78170819598
:1011A00084278523842781932F5F3F4F2530310586
:1011B00069F7089520E1929F800D1124682F6695AC
:1011C00066956695982F977085E0689FB001112409
:1011D00040E050E080E0FB01E40FF51FE453FE4FD8
:1011E000208130E0092E02C0369527950A94E2F757
:1011F00021703327042E01C0220F0A94EAF7822BB4
:101200004F5F5F4F4530510531F70895BF92CF9240
:10121000DF92EF92FF920F931F93CF93DF938C0196
:10122000C090FE01D090FF01E0900002F09001021A
:101230008091020290910302A0910402B0910502F4
:10124000C82AD92AEA2AFB2ACFE1D0E0D701C60171
:101250000C2E04C0B695A795979587950A94D2F75A
:1012600080FD04C0219790F7B12C07C0BC2EB801B7
:101270008C2F0E9455100197A9F38B2DDF91CF91F0
:101280001F910F91FF90EF90DF90CF90BF90089546
:10129000CF93DF93EC010E940609BE010E94551016
:1012A000DF91CF9108951F93CF93DF93EB0190913E
:1012B000CB01992321F0CB010E94480913C0882358
:1012C00049F0CB010E940609182F682FCE010E9419
:1012D000AF0804C0CB010E94DA08182FBE01812F8D
:1012E0000E945510DF91CF911F9108951F93CF93C6
:1012F000DF93C091060216E080910702C81799F0AB
:10130000D0E01C9FF0011D9FF00D1124E85FFD4F00
:101310004081518162817381848195810E948F0710
:101320002196C770E9CFDF91CF911F910895409129
:1013300038025091390260913A0270913B028091DB
:101340003C0290913D020C948F07EF92FF920F9315
:101350001F93CF93DF9380913D0282958F7009F0A8
:1013600065C080913A02882309F460C0809106022A
:10137000F0900702109138020091390260913B020F
:1013800070913C0291E01F3F09F090E0C091000194
:10139000D0910101292F96E0E92E8F1509F446C05E
:1013A0006115710521F00F3F21F030E003C031E0FD
:1013B00001C0322F90E030FD36C0E89EF001E99E7A
:1013C000F00D1124DF01A85FBD4F11963C911197DC
:1013D000301329C03C91311326C012963C911297CC
:1013E000311121C013964D915C911497461B570BF8
:1013F0004C175D07C0F480913D028F70806180932F
:101400003D02E35FFD4F80818F708061808388E3C0
:1014100092E00E940D07DF91CF911F910F91FF90F5
:10142000EF900C94760901968770B7CFDF91CF913A
:101430001F910F91FF90EF9008959F92AF92BF92EE
:10144000CF92DF92EF92FF920F931F93CF93DF9390
:10145000CDB7DEB761970FB6F894DEBF0FBECDBF34
:101460008C0185E0F801DE011D9601900D928A95B0
:10147000E1F7D8011296EC9090913802E091390290
:1014800020913B0230913C022115310531F0EF3FB4
:1014900031F481E09F3F19F403C081E001C080E096
:1014A000B82FB1709B2E80FD47C1D8014C91119689
:1014B0005C9111971396AD90BC90149788E3C82E59
:1014C00082E0D82EF0903A02B501621B730B209196
:1014D000000130910101FF2009F4D9C080913D0243
:1014E0006217730708F095C0282F207F09F052C0BB
:1014F0005E1313C0491311C0FE2CE1100EC08F7093
:10150000806180933D020E949709C6010E940D07E9
:1015100080913D02F80185834DC1AB2831F05F3FDA
:1015200031F481E04F3F19F403C081E001C080E055
:1015300080FD03C081E08E2502C080E090E0F82F9E
:10154000F170FF2E80FF1CC08091060220910702DF
:1015500036E0821709F40BC190E0389FF001399F03
:10156000F00D1124E85FFD4F6181561306C06081C4
:10157000461303C06281E61203C001968770E9CF6B
:10158000FE2CEE2009F416C180913D02816080930B
:101590003D0254C05E1306C0491304C0E11002C0EE
:1015A000F80199C0C8010E947807882361F1EE20F4
:1015B00051F120913D02822F82958F7090E0029729
:1015C00074F0809138029091390298878F83198640
:1015D000BB86AA862C87CE0107960E940D0786E05F
:1015E000F801A8E3B2E001900D928A95E1F70E941C
:1015F000A5090E9497090AC05E1711F1C8010E944F
:10160000780781112CC0C8010E940D07FF24F394B4
:10161000D1C0282F207F81F77A2DB98AA88A6E2D14
:1016200089890E94800788E392E00E940D0786E086
:10163000D6011D928A95E9F70E949709F12CBAC04C
:101640004913DCCFE110DACFF8018583C8010E948D
:101650000D0786E0D6011D928A95E9F7ABC0EE2012
:1016600091F220913D02822F82958F7090E0029737
:101670000CF4B5CF80913802909139029A83898316
:101680001B82BD82AC822E83CE010196A6CF62174B
:10169000730708F044C0FE2CEE2009F4B4CF5E13AB
:1016A00030C049132EC020913D0220FD21C0822F61
:1016B00082958F70482F50E041155105C9F0F8010F
:1016C00025834F30510541F08F5F982F9295907F81
:1016D000822F8F70892B8583C8010E940D0786E0B9
:1016E000F801A8E3B2E001900D928A95E1F73CC0C1
:1016F00086E0F801A8E3B2E001900D928A95E1F747
:1017000059C0C8010E947807811169CF80913D02BC
:10171000816080933D02C8010E940D074BC07A2D65
:10172000B98AA88A6E2D89890E94800786E0D60131
:101730001D928A95E9F718C0EE2009F464CFC8011C
:101740000E947807F82E882309F45DCF86E0F8011F
:10175000A8E3B2E001900D928A95E1F788E392E068
:101760000E9406040E94A5090E94970923C04D8784
:101770005E878D859E850E944809292F22952F70AE
:10178000223028F49F7039F0811105C00BC024303D
:1017900028F49F7049F4805E883020F0C8010E94D0
:1017A0000D079F2CF92C06C0D80115969C91907FAF
:1017B00091F7F8CF8F2D61960FB6F894DEBF0FBE6C
:1017C000CDBFDF91CF911F910F91FF90EF90DF90F0
:1017D000CF90BF90AF909F9008951F93CF93DF93CA
:1017E000CDB7DEB72C970FB6F894DEBF0FBECDBFD6
:1017F0004F83588769877A878B879C87CE010796A6
:101800000E941D0A8823D1F09F8188852A853B8507
:10181000232B31F08F3F31F481E09F3F19F403C057
:1018200081E001C080E080FD47C04F815885698517
:101830007A858B859C850E948F073EC086E0FE01DD
:101840003796DE01119601900D928A95E1F7FF819E
:10185000E8856A857B856115710531F0EF3F31F4CC
:1018600081E0FF3F19F403C081E001C080E080FD0A
:1018700023C02091070230E0C901019687709927A3
:101880004091060250E084179507F1F1F983EA834D
:101890007D836C8396E0929FD001939FB00D1124BD
:1018A000A85FBD4FFE01319601900D929A95E1F728
:1018B000809307020E94760916E0809106029091BB
:1018C0000702891771F1189FC0011124885F9D4F8D
:1018D0000E941D0A882329F1E09106021E9FF00153
:1018E0001124E85FFD4F40815181628173818481C1
:1018F00095810E948F078091060290E00196877083
:10190000992780930602D9CF0E94590710920702A7
:1019100010920602E8E3F2E086E0DF011D928A956C
:10192000E9F72C960FB6F894DEBF0FBECDBFDF915E
:10193000CF911F91089580915E028595859585953B
:10194000089580915E028770089590915E0297706D
:1019500081E009F480E008958091810208959091DA
:101960008102892B80938102089580959091810254
:1019700089238093810208951092810208959091A5
:101980008002892B80938002089580959091800237
:101990008923809380020895109280020895809197
:1019A0005F02089508950C94D20C0C94D30C90917E
:1019B000E30292FD08C090915F02981721F0809396
:1019C0005F020C94D50C089580915F02882329F062
:1019D00010925F0280E00C94D50C0895CF93DF93B2
:1019E000E0910201F0910301809181028083E091F6
:1019F0000201F0910301908180918002892B808304
:101A000080915F02882381F0E0910201F09103014F
:101A10009081892B808380910201909103010E9423
:101A2000122181110E94E40CC0910201D0910301A6
:101A300040E250E06EE372E0CE010E94762A892BEC
:101A400069F080E2FE01AEE3B2E001900D928A956A
:101A5000E1F7CE01DF91CF910C94BE20DF91CF91C1
:101A600008950C94D20C9091E30292FD10C098E07E
:101A7000899F90011124262B20935E020E94110859
:101A800080915E028595859585950C94310D0C9419
:101A9000110810925E0280E00C94310D20915E02DC
:101AA0008095822380935E02982F977099F430E09E
:101AB000482F082E000C550B2417350759F090912C
:101AC000E30292FD07C08595859585950E943208B1
:101AD0000C94490D08959091E30292FB222720F97E
:101AE000281769F080FB92F99093E3028091E2025B
:101AF0009091E3020E94B30D82E00C944E0D089584
:101B00008091E30282FB882780F991E089270C9479
:101B10006B0D81E00C946B0D80E00C946B0D80E0FC
:101B200090E00E94912A21E0893E9E4F09F020E03A
:101B3000822F089582E090E00C94832A83E090E065
:101B40000C94832ACF9384E090E00E94832AC82FCC
:101B500082E290E00E94832A2C2F30E0A901582BCA
:101B6000CA01CF910895CF93C92F682F84E090E0E8
:101B70000E94972A6C2F82E290E0CF910C94972AD2
:101B8000AB01BC018FE090E00C94A92AAB01BC0131
:101B900083E190E00C94A92A60E070E0CB010C9402
:101BA000C60D60E070E0CB010E94C00D0C94CC0D1E
:101BB00069EE7EEF80E090E00E94B52A60E082E06E
:101BC00090E00E94972A60E083E090E00E94972ACC
:101BD0001092020210920302109204021092050267
:101BE00060E084E090E00E94972A60E082E290E06A
:101BF0000E94972A60E085E090E00E94972A60E0CA
:101C000086E090E00E94972A6FEF87E090E00E94C4
:101C1000972A40E050E0BA0188E090E00E94A92AAB
:101C200060E08DE090E00E94972A40E050E0BA0129
:101C300088E190E00E94A92A60E087E190E00E949C
:101C4000972A40E050E0BA018CE190E00E94A92A76
:101C500060E070E080E290E00E94B52A40E050E051
:101C6000BA0188E190E00E94A92A0C94D10D0C944D
:101C7000D80D682F8EE090E00C94972A0E9478226D
:101C800060939002709391028093920290939302DA
:101C900060938C0270938D0280938E0290938F02DA
:101CA000089585B7806885BF85B7806885BF08952A
:101CB00081E008950C94580E08950C945C0E0C94D9
:101CC0005C0E0C945F0E0C945C0E0C94630E0C94E2
:101CD0005C0E0E94510E81E391E10E94A8200E94B7
:101CE000670E0C94650E0E945D0E0C945C0E0E94B3
:101CF00034110E949E030C942F1E0E9463220E94A6
:101D000019120E94770E0E94681C0E94A71A0C9458
:101D1000610E5F926F927F928F929F92AF92BF926D
:101D2000CF92DF92EF92FF920F931F93CF93DF93A7
:101D3000CDB7DEB72A970FB6F894DEBF0FBECDBF82
:101D40000E942E12C82E81110E943E0E32E8832E70
:101D500032E0932E00E010E0502E802F0E945811A8
:101D60005C01F401619071904F016826792661143D
:101D70007104B1F40F5F1F4F0530110569F78FEF44
:101D800089838A831B820E946C228160782F9D83C5
:101D90008C8349815A816B818D810E94BC033AC03A
:101DA0008091940281FD0E946111D12CEE24E39474
:101DB000F12CC3018E219F21892B29F10E945A0EFB
:101DC0008823A9F0DE825F82AE20BF2081E0AB28AD
:101DD00009F480E088870E946C228160782F9A87BE
:101DE00089874E815F8168858A850E94BC03000FC8
:101DF000111FF801EE57FD4F80819181E826F926E9
:101E0000F182E08207C0D394EE0CFF1CF0E1DF12F8
:101E1000D0CFB0CF81E0C11001C080E02A960FB6CC
:101E2000F894DEBF0FBECDBFDF91CF911F910F9110
:101E3000FF90EF90DF90CF90BF90AF909F908F90EA
:101E40007F906F905F9008950E94890E0E94DA1A29
:101E50000E942E1E0E9435140C94B103CF93DF9381
:101E60000E945A10EC01811521E5920708F045C047
:101E7000811530E5930708F094C0883E910528F558
:101E8000803E910508F0F8C0883A910570F4853AD3
:101E9000910508F07CC08130910509F475C008F403
:101EA000E8C0049708F0E8C0E4C08F3B910508F053
:101EB000E0C0C85AD0E0CC0FDD1FC35ADE4F0990F6
:101EC000D881C02DCE019464D8C0811540E294071A
:101ED00058F4811551E0950708F0CEC08D3E91056C
:101EE00008F4C7C09065C9C0C11580E4D80708F4DC
:101EF000C0C0DF70CE01906AC0C0811525E5920791
:101F0000A8F4811534E5930708F095C0811543E5E1
:101F1000940708F07BC0811552E5950708F061C071
:101F2000D82FCC27CE01816F906AA7C0C11589E553
:101F3000D807A0F4C11528E5D20708F082C0C11562
:101F400036E5D30708F095C08C2F0E94EE108F71F4
:101F500090E0D82FCC27CE0190628FC0C1154AE502
:101F6000D40708F474C0CE0190568115904208F051
:101F700080C08D2F8F710E94EE10DD27D0628F718F
:101F8000AE01582BCA0179C081E090E076C0C55AF5
:101F9000D0E0C557DE4F8881C82FD0E0CE019064D5
:101FA0006CC074E0969587957A95E1F7282F237099
:101FB0003C2F337081E090E002C0880F991F3A9562
:101FC000E2F79C68AC01522B9A019C2F9F7096956A
:101FD000969550E2959FE0011124C9018C2B9D2B11
:101FE0004CC08370992721E030E002C0220F331FDC
:101FF0008A95E2F79C2F9695969580E2989FE0014E
:102000001124C22BD32BCE019C6837C08370992733
:1020100021E030E002C0220F331F8A95E2F79C2FA7
:102020009695969540E2949FE0011124C22BD32B04
:10203000CE019A6822C0D82FCC27CE01846F906A37
:102040001CC0DC2FCC27CE01806F906A16C08C2F6D
:102050008F700E94EE1094E0D695C7959A95E1F79F
:10206000CF70D0E0DC2FCC27D0699E01282BC9018E
:1020700004C080E090E001C0CE01DF91CF910895CF
:10208000E72FF0E095E0899FE00DF11D112484E039
:10209000EE0FFF1F8A95E1F7E60FF11DEE0FFF1F10
:1020A000E852FF4F8591949108950E9440100E943C
:1020B0002E0F08958238910569F1B0F481339105AE
:1020C00009F46DC048F48932910509F463C08A327D
:1020D000910509F469C008958533910509F455C047
:1020E00089339105B9F00895833E910569F138F47B
:1020F000803E9105B1F0823E910509F10895863E3A
:102100009105A9F1873E9105B9F1843E910509F049
:1021100064C023C02091E20220FD4FC021FD4DC0CC
:1021200008958091E20280FD44C08091E30280FF27
:1021300044C08091E20284FD42C083EE4DC0809194
:10214000E20282FF38C0F5CF8091E20282FD33C007
:102150008091E30280FD31C0ECCF8091E30281FFEA
:1021600032C08091E20284FD2AC087EE35C08091A2
:10217000E20283FF26C0F5CF8091E20283FD21C0F9
:102180008091E30281FD1FC0ECCF8091E20285FDCA
:102190001CC01DC08091E20285FD19C016C080914F
:1021A000E20286FD16C017C08091E20286FD13C0D0
:1021B00010C089E311C082EE0FC080EE0DC080E038
:1021C0000BC086EE09C084EE07C089E205C085E336
:1021D00003C08AE201C081E390E008959091E20299
:1021E00092FF0DC0282F2871283019F4877F846052
:1021F00006C0282F2471243011F48B7F886093FF50
:102200000DC0282F2871283119F4877E846106C0FB
:10221000282F2471243111F48B7E88612091E302F0
:1022200020FF0DC0382F3871383019F4877F816056
:1022300006C0382F3171313011F48E7F886021FF54
:102240000DC0282F2871283119F4877E816106C0BE
:10225000282F2171213111F48E7E886194FD877EB3
:10226000089580E0089508950E948F0D811102C0A5
:102270000E94370E0E949A0D809394020E94A20D34
:102280009093E3028093E2020E9433110E949E0D1C
:10229000682F70E080E090E00E94B1076091FE013D
:1022A0007091FF0180910002909101020C94E90766
:1022B000E82FF0E0EE0FFF1FE251FD4F808191818A
:1022C0000895089580EA8A95F1F7089500C0089569
:1022D0000C94621108950C946A110C946B110C9477
:1022E0006A110C946F11F894E82FE295EF70F0E00A
:1022F00031A1282F2F7081E090E001C0880F2A952E
:10230000EAF7982F9095932391A392A1892B82A30A
:10231000789408950F931F93CF93DF93CEE9D1E084
:1023200089918F3F11F00E94731181E0C33AD80761
:10233000B9F7CEE8D1E00EE911E089918F3F11F0B5
:102340000E9473110C171D07C1F7DF91CF911F91E8
:102350000F910895BF92CF92DF92EF92FF920F9369
:102360001F93CF93DF938C01C62FD0E0CE0182560E
:102370009E4F6C01FC0190819F3F09F450C0B62E26
:10238000F894E92FE295EF70F0E081A19F7021E0D1
:1023900030E001C0220F9A95EAF7822B81A382A137
:1023A0002095282322A378940E946611EEE8F1E09C
:1023B0004EE951E021E030E0E12CF12C61916F3FDA
:1023C00089F0A62FA295AF70B0E090968C9190E026
:1023D0006F7002C0959587956A95E2F780FD02C0FF
:1023E000C90102C080E090E0E82AF92A220F331FD9
:1023F0004E175F0719F7F60180818F3F11F00E9499
:10240000731161E0E114F10409F460E08B2D0E9486
:102410006811CC0FDD1FC00FD11FF982E882DF9158
:10242000CF911F910F91FF90EF90DF90CF90BF90D1
:1024300008950E948A118AE0EEEEF2E0DF01982F03
:102440001D929A95E9F7E4EEF2E0DF011D928A957C
:10245000E9F785E00E9479120C940B03FF920F9329
:102460001F93CF93DF93CDB7DEB72A970FB6F894BB
:10247000DEBF0FBECDBF8E010F5F1F4F8AE0F80198
:1024800011928A95E9F7F12C6F2DC8010E94AA11CB
:10249000F394F5E0FF12F8CF4AE050E0B80184EE83
:1024A00092E00E94762AFF24F394009709F4F12C1D
:1024B000892B41F08AE0F801A4EEB2E001900D9280
:1024C0008A95E1F72F2D45E06EEE72E084EE92E002
:1024D0000E947A120E940D038F2D2A960FB6F8944F
:1024E000DEBF0FBECDBFDF91CF911F910F91FF9047
:1024F00008950895FF920F931F93CF93DF93F82EC3
:10250000092F162FD72FC42F222349F081E0809363
:1025100097020E946C22909396028093950280917C
:1025200097028823D9F080919502909196020E949B
:102530008422059798F0EF2DF02FA12FBD2F80E07A
:1025400090E04C2F50E08417950734F4219131919D
:102550002D933D930196F7CF10929702DF91CF9183
:102560001F910F91FF9008950E9484240E947D0E78
:102570000C9490240E9494240E94240F0C94AE2466
:102580000E940A220E946B240E94690E0E94B412CB
:102590000E94BA120E94730EFBCF80919E0280FFB0
:1025A00006C06091090170E0660F771F26C081FFA9
:1025B00004C06091090184E005C082FF07C06091FA
:1025C000090188E0689FB001112417C090919D0215
:1025D0009923D1F060910801961788F7209109019D
:1025E00088E0289F90011124929FA001939F500D95
:1025F000112470E0CA010E94F0296038710540F48E
:102600006115710519F406C068E070E0862F089521
:102610008FE7089581E0089580919E0280FF08C0B1
:102620006091050170E0759567957595679521C076
:1026300081FF06C06091050170E07595679519C02E
:1026400082FF04C06091050170E010C090919C026F
:10265000992399F0609104019617A0F780910501E4
:10266000899FC001112470E00E94F0296038710533
:1026700040F46115710519F406C061E070E0862F21
:1026800008958FE7089581E008958D3E21F40E941A
:10269000CD12819504C08E3E29F40E94CD12809304
:1026A000A20208958F3E21F40E94CD12819504C0AC
:1026B000803F29F40E94CD128093A1020895893FA2
:1026C00019F40E940C1305C08A3F31F40E940C13C8
:1026D00081958093A30208958B3F21F40E940C13EF
:1026E000819504C08C3F29F40E940C138093A402AE
:1026F00008959FE0980F983078F421E030E0A90128
:1027000002C0440F551F9A95E2F7CA019091A002AA
:10271000892B8093A00208958D3F21F480919E0221
:1027200081600BC08E3F21F480919E02826005C0C3
:102730008F3F29F480919E02846080939E020895C9
:102740008D3E39F49091A20297FF35C01092A202FB
:1027500059C08E3E29F49091A2021916BCF32BC0E9
:102760009091A1028F3E29F497FF25C01092A102FB
:1027700049C0803F19F41916CCF31DC09091A302F3
:10278000893F29F41916BCF41092A3023BC08A3F7A
:1027900019F497FF10C0F8CF8B3F39F49091A40241
:1027A00097FF09C01092A4022DC08C3F21F4909194
:1027B000A4021916BCF39FE0980F983080F421E032
:1027C00030E0A90102C0440F551F9A95E2F7CA01F3
:1027D00080959091A00289238093A00213C08D3F21
:1027E00021F480919E028E7F0BC08E3F21F4809158
:1027F0009E028D7F05C08F3F29F480919E028B7FC2
:1028000080939E028091A102811106C08091A20254
:10281000811102C010929D028091A302811106C015
:102820008091A402811102C010929C0208950E941E
:102830006C222091A102211104C02091A202222326
:1028400021F090939B0280939A022091A302211180
:1028500004C02091A402222321F090939902809336
:1028600098028FE992E00C94D820EF92FF920F9398
:102870001F93CF93DF9300D000D000D0CDB7DEB749
:1028800086E0EFE9F2E0DE01119601900D928A9563
:10289000E1F7E090A102F090A2020091A302109152
:1028A000A4021092A1021092A2021092A30210920E
:1028B000A402E11003C0FF2009F45DC080919A02D8
:1028C00090919B020E948422AC0190919D029923D9
:1028D00039F020910A0130E02417350758F04BC039
:1028E00020910B018AE0289F9001112424173507BD
:1028F00018F041C09F3F19F09F5F90939D02EE201A
:1029000061F00E94CD121E1414F09FEF01C091E0FF
:10291000989F902D11249093A102FF2061F00E94B6
:10292000CD121F1414F09FEF01C091E0989F902DDD
:1029300011249093A2023091A1023323E1F020915F
:10294000A2022223C1F045EB3403C00111249923D4
:1029500019F09093A10203C081E08093A10235EBAE
:102960002303C0011124992319F09093A20203C0FC
:1029700081E08093A202011103C0112309F45DC01C
:1029800080919802909199020E948422AC019091CA
:102990009C02992339F02091060130E02417350775
:1029A00058F04BC0209107018AE0289F9001112424
:1029B0002417350718F041C09F3F19F09F5F90938F
:1029C0009C02002361F00E940C13101614F09FEF7C
:1029D00001C091E0989F902D11249093A3021123A0
:1029E00061F00E940C13111614F09FEF01C091E0EA
:1029F000989F902D11249093A4023091A302332329
:102A0000E1F02091A4022223C1F045EB3403C00180
:102A10001124992319F09093A30203C081E08093BD
:102A2000A30235EB2303C0011124992319F09093DD
:102A3000A40203C081E08093A4028091A1028111CD
:102A40000BC08091A202811107C08091A302811165
:102A500003C08091A40281110E941714EB82FC82B2
:102A60000D831E8386E0FE013196AFE9B2E001904E
:102A70000D928A95E1F726960FB6F894DEBF0FBE49
:102A8000CDBFDF91CF911F910F91FF90EF900895EF
:102A9000EFE9F2E086E0DF011D928A95E9F71092F6
:102AA0009D0210929C0210929E020895EF92FF9256
:102AB0000F931F93CF93DF938B01682F11110AC0DF
:102AC000442329F0E82FF0E0E157FD4F6491762F81
:102AD000862F75C0212F30E0E82FF0E0442321F04D
:102AE000E157FD4FE491F0E046E0049FC00111245E
:102AF000CFEFD0E0BE010E94DC294BEA4603C001C3
:102B0000479F900D1124800F911D800F911D982FCC
:102B1000990F890FAE01421B530B4E9FD0014F9F5F
:102B2000B00D5E9FB00D11249B2F189FA0011124A2
:102B3000452F55278E01041B150B0E9FA0010F9FDB
:102B4000500D1E9F500D11247E01E81AF108E29EDF
:102B50008001E39E100DF29E100D1124212F3327CA
:102B6000C21BD30BCE9F9001CF9F300DDE9F300D47
:102B7000112462307105A9F048F46115710569F0FE
:102B800061307105C9F48B2F752F0DC0643071054C
:102B900081F058F06630710579F47E2F8B2F932FDA
:102BA0000DC0832F7B2F9E2F09C08E2F7B2F952F3B
:102BB00005C08E2F732F02C07E2F852F692FDF91C6
:102BC000CF911F910F91FF90EF90089541E00E94E7
:102BD0005615089508950E94E6150895CF93DF9342
:102BE000762FE901682F842F0E94EB157983688383
:102BF0008A83DF91CF9108958091F802282F26953E
:102C000030E02115310519F48170826005C025324C
:102C1000310524F0817088648093F802089588E07B
:102C200090E00C948B2ACF92DF92EF92FF926B018F
:102C30007C010E94FC15B701A60188E090E0FF909E
:102C4000EF90DF90CF900C94A92AE8EFF2E083E0B8
:102C5000808311828FEF82838383148260817181EC
:102C6000828193810C9413168091F80280FF02C038
:102C70008695089580E008959091FC02933018F4B1
:102C80009F5F9093FC02882351F06091F80270914D
:102C9000F9028091FA029091FB020C9413160895A8
:102CA00081E00C943C169091FC02992319F091500C
:102CB0009093FC02882351F06091F8027091F90220
:102CC0008091FA029091FB020C941316089581E012
:102CD0000C94531670E00C943F1E6091100180918B
:102CE000F80280FF0AC080910F0123E0829FC0019B
:102CF000112483509D4F0C946A168091110190917C
:102D00001201891780F7E82FF0E09F01220F331F8F
:102D1000E20FF31FE350FD4F1182108212828F5F8A
:102D2000F0CF9091F80290FF16C090911101209180
:102D30001201921770F4E92FF0E0DF01AA0FBB1F18
:102D4000EA0FFB1FE350FD4F8183608342839F5F47
:102D5000F0CF0C946D160895CF93DF9300D01F929F
:102D6000CDB7DEB79091F80290FF0AC09E012F5FA9
:102D70003F4F0E94EE154B8169818A810E94911616
:102D80000F900F900F90DF91CF910895CF93DF9325
:102D9000EC01EC81F0E0E657FE4F4491E8EFF2E001
:102DA000628181810E94AC168C818F5F8C83DF9160
:102DB000CF910895CF93DF93EC01E8EFF2E04381E8
:102DC00062818C810E94AC168C818F5F8C83DF9135
:102DD000CF9108950F931F93CF93DF9300D01F924D
:102DE000CDB7DEB78C018091A50281110AC09E018A
:102DF0002F5F3F4F4FEF6FEF0E94EE158A81809358
:102E0000A502F8018481813051F028F0823061F40C
:102E10004091A5020AC08091A50240E007C06091E0
:102E2000A50240E080E003C040E080E060E00E9456
:102E30009116F801848190E0019663E070E00E94B1
:102E4000F02984830F900F900F90DF91CF911F9105
:102E50000F910895AF92BF92CF92DF92EF92FF92BF
:102E60000F931F93CF93DF9300D01F92CDB7DEB7A0
:102E7000182FF62E042FE22E9091F80290FF6DC0CD
:102E8000E92FE695AE2FB0E0AD55BE4F8C91809303
:102E9000AF029E7F923061F49E012F5F3F4F812FE2
:102EA0000E94EE154B8169818A810E94911643C070
:102EB000823019F40091FB023EC0863019F4109163
:102EC000F90239C08930D9F38931A9F5E9518E2F3A
:102ED0008170D82EE695F0E0E657FD4FA590B490AE
:102EE000C12CBB2460911301C61618F52C2D30E0BF
:102EF000A29EC001A39E900DB29E900D112470E081
:102F00000E94DC29812FD11002C0860F01C0861BD0
:102F100090911101290F311DA901440F551F240F54
:102F2000351F23503D4F402F6F2D0E94EE15C39447
:102F3000D9CF0E946D161093F902F092FA02009315
:102F4000FB02EE2051F06091F8027091F90280913D
:102F5000FA029091FB020E9413160F900F900F90AF
:102F6000DF91CF911F910F91FF90EF90DF90CF9065
:102F7000BF90AF900895E8EFF2E09181282F438150
:102F8000628188E0890F0C942A1781E00C94BB17AA
:102F9000E8EFF2E09181282F4381628188EF890F69
:102FA0000C942A1781E00C94C817E8EFF2E06281D4
:102FB00028E0620F08F46FEF282F438181810C9481
:102FC0002A1781E00C94D517E8EFF2E0628128E03F
:102FD000621B08F460E0282F438181810C942A173A
:102FE00081E00C94E417E8EFF2E0438128E0420F1F
:102FF00008F44FEF282F628181810C942A1781E019
:103000000C94F317E8EFF2E0438128E0421B08F448
:1030100040E0282F628181810C942A1781E00C9472
:10302000021820E00C942A17FF920F931F93CF935E
:10303000DF93EC01F12C0FEF10E060911301F61615
:10304000F0F4809111012F2D30E0280F311DC901BE
:10305000880F991F280F391F23503D4F70E0C8017A
:103060000E94F029962F8C814091FB026091FA0218
:10307000F99E800D11240E94EE15F394DECF0E947C
:103080006D169A818C8190FF02C08F5F01C08150C4
:103090008C83DF91CF911F910F91FF900895AF9294
:1030A000BF92CF92DF92EF92FF920F931F93CF9335
:1030B000DF93FC01828180FF02C00FEF01C001E0BD
:1030C00010E044E1A42E80911301181708F043C0CA
:1030D00080911101C12ED12CE601C80FD11DCE0166
:1030E000880F991FC80FD91FC350DD4F198218824E
:1030F0001A8234E0E32EF12CB12C8091A7028B0DC3
:1031000085312CF06A2D0E94CE29892F05C087FFBA
:1031100003C090911301890F082E000C990BC8165B
:10312000D90691F48091FB028E9DA0018F9D500DD8
:10313000112455954795559547959E016091FA0242
:103140008091F9020E94EE15B00EF1E0EF1AF1083D
:10315000A1F61F5FB8CF0E946D168091A7020130C3
:1031600031F4811102C080911301815007C090E0B9
:1031700001966091130170E00E94F0298093A702EC
:10318000DF91CF911F910F91FF90EF90DF90CF9043
:10319000BF90AF900895CF9380911101909112014B
:1031A000891770F4E82FF0E09F01220F331FE20F20
:1031B000F31FE350FD4F1182108212828F5FF0CF18
:1031C000C0E060911301C617C0F5EC2FF0E070E08D
:1031D000CF010E94F02920911101820F2091A602B7
:1031E000022E000C330B90E0E217F307CCF0209195
:1031F0000E01022E000C330B2E173F078CF09C01A2
:10320000220F331F820F931F9C0123503D4F40918B
:10321000FB026091FA028091F9020E94EE150BC048
:10322000FC01EE0FFF1F8E0F9F1FFC01E350FD4FAF
:10323000118210821282CF5FC4CF0E946D1620913E
:103240000D018091A602820F8093A60290910E013B
:10325000920F90930E0119165CF4082E000C990B36
:103260004091130150E041505109841795071CF01B
:10327000219520930D01CF9108958F929F92AF9247
:10328000BF92CF92DF92EF92FF920F931F93CF9353
:10329000DF938C01FC014481C42FD0E09E01DE014C
:1032A0000E94342A9B01AC010E944A2A6B017C01D6
:1032B000E0E2F0E0EC1BFD0BA5E5B0E09B01AC010A
:1032C0000E944A2A4B015C019F01DF010E942C2AC7
:1032D0009B01AC010E94552A9B01AC012C0D3D1DA8
:1032E0004E1D5F1DC501B4010E94042AC22FD22FBA
:1032F0002A3228F4F3E02F9F900111240DC025E518
:1033000030E02C1B3109C901880F991F280F391F84
:1033100037FF02C02F5F3F4F35952795C22FC095CD
:10332000F12C85E5E82EED1A80911301F816C8F40A
:10333000F1FC02C08E2D01C08D2F909111012F2D17
:1033400030E0290F311DA901440F551F240F351FEF
:1033500023503D4F4C2F6091FA020E94EE15F394DA
:10336000E3CF0E946D16F8018481811102C091E0C3
:1033700003C0803219F49FEF90930C0190910C01DF
:10338000890FF8018483DF91CF911F910F91FF90F6
:10339000EF90DF90CF90BF90AF909F908F90089567
:1033A0000F931F93CF93DF93EC0100E010E0809127
:1033B0001301282F30E00217130724F59091110113
:1033C0009801290F311DA901440F551F240F351FE6
:1033D00023503D4F869590E04C81081719071CF447
:1033E000442331F002C0411103C04091FB0201C0EF
:1033F00040E06091FA028091F9020E94EE150F5FA1
:103400001F4FD5CF0E946D168C8190E00196817080
:1034100099278C83DF91CF911F910F910895E8EF49
:10342000F2E080818E7F80836081718182819381CF
:103430000E9413161092B0022FEF80E792E0215005
:1034400080409040E1F700C000000C946D16609140
:10345000F802669570E04BE050E084E191E00E9454
:10346000692A892B19F481E08093B0020E946C22B2
:103470009093A9028093A80208959091F80290FF7A
:1034800035C09170811102C0926006C0853210F083
:10349000986402C0880F982B9093F802662351F02D
:1034A0006091F8027091F9028091FA029091FB020A
:1034B0000E9413166091F802669570E04BE050E0B0
:1034C00084E191E00E94692A892B19F01092B002E0
:1034D00002C00E94271A81E08093AB024091FB0258
:1034E0006091FA028091F9020C9411180895682FE6
:1034F0009091F802969581E0890F853208F081E07D
:103500000C943D1A81E00C94771A682F9091F80280
:1035100096958FEF890F09F484E20C943D1A81E0AF
:103520000C94851A61E00C943D1AE8EFF2E080817A
:103530008160808386950C94921A8091F80280FDB8
:103540000C940F1A0C94951A60E00C943D1A80911B
:10355000AE0281112EC00E948F0D811104C00E9405
:10356000370E0E9425160E940F166093F802709382
:10357000F9028093FA029093FB026E7F61F40E943D
:1035800025160E940F166093F8027093F90280933B
:10359000FA029093FB020E94FC151092B0028091F7
:1035A000F80280FF03C086950E94A41A81E08093F0
:1035B000AE0208950F931F93CF93DF938091B002D3
:1035C000882309F485C08091AF02E091F802E69566
:1035D000E81BE093AA02823049F4F0E0EA57FE4F7C
:1035E000E491CE2FD0E006EC16E149C0863049F4D4
:1035F000F0E0ED57FE4FE491CE2FD0E00AED16E15A
:103600003EC0893051F4E695F0E0E058FE4FE49179
:10361000CE2FD0E004E118E132C08F3051F4E695AE
:10362000F0E0E358FE4FE491CE2FD0E00FE418E134
:1036300026C0853149F4F0E0E658FE4FE491CE2FE4
:10364000D0E00BEC18E11BC0883181F0833239F4F3
:10365000E8E7F1E0C591D4910AEE16E110C084329A
:1036600051F4C4EFD1E000ED19E109C0C8E2D0E0A7
:103670000DE319E104C0C0EDD7E00AEE15E1809139
:10368000AB02882361F01092AB020E946C229093EF
:10369000A9028093A8021092AD021092AC020E947F
:1036A0006C22E091A802F091A9028E1B9F0B8F3F24
:1036B0009F4770F4EC0FFD1FF093A902E093A8025E
:1036C00088EA92E0F801DF91CF911F910F91099460
:1036D000DF91CF911F910F910895882311F0FA0186
:1036E00001C0FB010994CF93DF93C82FD62F0E940E
:1036F00034168C1740F00E9434168D1720F4DF9199
:10370000CF910C94821A8C2FDF91CF910C94921A46
:103710001F93CF93DF93FB0112811111C3C0EC0102
:103720000E94AC0C8272CD3CFCE5DF0709F49AC024
:10373000A8F5C73CECE5DE0709F476C0A8F4C43C64
:103740009CE5D90709F45FC028F4C33CDC4509F4C3
:1037500057C054C0C53C9CE5D90709F459C0C63CC4
:10376000DC4509F45CC04AC0CA3CFCE5DF0709F44B
:103770006AC050F4C83CECE5DE0709F45AC0C93C05
:10378000DC4509F45BC03AC0CB3C9CE5D90709F4A1
:103790005FC0CC3CDC4509F460C030C0C23DFCE5F4
:1037A000DF0709F46FC088F4CF3C9CE5D90709F422
:1037B00060C008F45CC0C03DFCE5DF0709F45CC0F4
:1037C000C13DDC4509F45BC019C0C53D9CE5D90786
:1037D00009F460C050F4C33DFCE5DF0709F455C0AF
:1037E000C43DDC4509F454C009C0C63D9CE5D90779
:1037F00009F455C0CE35DD4509F454C011E052C07E
:103800000E949D1A4FC04FE85AE162E87AE104C075
:1038100042E85AE16FE87AE10E946D1B43C042ED35
:1038200057E165EC77E1F8CF45EC57E162ED77E1E0
:10383000F3CF40EF57E161EE77E1EECF41EE57E194
:1038400060EF77E1E9CF4EE058E16FEF77E1E4CF49
:103850004FEF57E16EE078E1DFCF47E656E160E5F4
:1038600076E1DACF40E556E167E676E1D5CF81E053
:1038700017C065E082E010C068E086E00DC06EE031
:1038800089E00AC064E18FE007C067E185E104C018
:1038900088E106C062E289E10E94731B03C083E2F3
:1038A0000E94921A812FDF91CF911F91089586E097
:1038B00090E00C94832A682F86E090E00C94972A7D
:1038C0008091390384708961809339030C945B1C67
:1038D0000E948F0D811104C00E94370E0E94601C4F
:1038E0000E94571C80933903282F269526952695EC
:1038F00030E02430310524F08770886180933903EB
:103900008091390380FF04C086958695869501C015
:1039100080E00C94791D20913903822F869586953D
:103920008695482F50E04330510554F48F5F982F0F
:10393000990F990F990F822F8770892B80933903E4
:10394000809139038160809339030E945B1C8091D0
:1039500039038695869586950C94791D8091390357
:10396000982F969596959695A1F0915E990F990F3F
:10397000990F8770892B80933903887F91E009F430
:1039800090E08091390390FB80F9809339030E9485
:103990005B1C809139038695869586950C94791DDC
:1039A0008091390380FD13C0816080933903813099
:1039B00019F489E080933903809139030E945B1CDC
:1039C000809139038695869586950C94791D089586
:1039D0008091390380FF08C08E7F809339030E9455
:1039E0005B1C80E00C94791D08958091390380FD63
:1039F0000C94E81C0C94D01C90913903892F869567
:103A0000869586958F5F8F719770843038F4880F14
:103A1000880F880F892B8093390302C09093390354
:103A200080913903887F91E009F490E08091390317
:103A300090FB80F9809339030E945B1C80913903CD
:103A40008695869586950C94791D843008F083E0E0
:103A5000909139039770282F220F220F220F922B5B
:103A600090933903987F21E009F420E09091390385
:103A700020FB90F9909339030C94791D0E94251D29
:103A8000809139030C945B1C9C01FB01828188238B
:103A900049F12E3BFCE53F07C9F040F42C3BECE537
:103AA0003E0769F02D3B3C4561F00895203C9CE5C4
:103AB000390791F070F0213C3C4589F0089583E08E
:103AC00001C080E00E943E1D80E008950E94AE1C6F
:103AD000FBCF0E948B1CF8CF0E94F51CF5CF0E94F3
:103AE000FC1CF2CF81E00895269A2E9808952E9816
:103AF00008958F929F92AF92BF92CF92DF92EF92F2
:103B0000FF920F931F93CF93DF93C82F843050F40D
:103B1000811109C0809180008F7D809380000E9478
:103B2000771D06C0C3E08091800080628093800092
:103B3000A0918600B09187002C2F30E00E94342A9B
:103B400023E030E040E050E00E94042A0027122FDA
:103B5000232F342F012F122F232F332780918600FC
:103B6000909187006CE070E00E94DC29601771077B
:103B700030F0C80169E070E00E94DC295EC08091ED
:103B8000860090918700E0908600F0908700E09199
:103B90008600F0918700C6E0D0E0BE010E94DC29DB
:103BA000060F171F211D311D4801590185E0880CA2
:103BB000991CAA1CBB1C8A95D1F7C701BE010E94A3
:103BC000DC296F01E12CF12CA7019601260F371F8C
:103BD000411D511DC501B4010E94042A69017A01E9
:103BE000E0918600F0918700CA01B9010E94BE29C8
:103BF0009B01AC01DF010E944A2A9B01AC01C70175
:103C0000B6010E94BE29DC01CB012FE0B695A79535
:103C1000979587952A95D1F7009186001091870096
:103C200020E030E0081719072A073B0728F46091C5
:103C3000860070918700CB01BC0170938B0060936C
:103C40008A00DF91CF911F910F91FF90EF90DF904D
:103C5000CF90BF90AF909F908F90089508950E944D
:103C6000741D82E28093800089E1809381008FEF50
:103C70009FEF90938700809386000C94681C6A9A4B
:103C80002EB12B7F3EB134604FB7F894FC01CB01CD
:103C9000880F991F680F791F6E0F7F1FE617F707B0
:103CA00089F0819198E03EB9000000C087FF2EB9ED
:103CB000880F000000C000C000C02EB900C09A9557
:103CC00091F7ECCF4FBF8FE594E00197F1F700C07B
:103CD00000000895CF93DF93EC01FB0182818823DC
:103CE00009F43CC1C430FDE5DF0760F4CB3F9CE53F
:103CF000D90788F49E0122503C452431310508F053
:103D00002EC109C0C236EDE5DE0729F0C63AFDE551
:103D1000DF0709F024C10E94A20D9093E302809373
:103D2000E202C1318CE5D80709F4C6C008F042C0F0
:103D3000C930ECE5DE0709F49BC000F5C5308CE521
:103D4000D80709F485C078F4C330ECE5DE0709F440
:103D500078C008F07AC0C230DC4509F0F5C0809127
:103D6000E2028160EFC0C7309CE5D90709F478C052
:103D700008F07AC08091E2028061E4C0CD30FCE5B9
:103D8000DF0709F487C058F4CB309CE5D90709F464
:103D900079C008F07BC08091E20288606FC0CF30AC
:103DA000FCE5DF0709F480C008F082C08091E202E0
:103DB000877FC8C0CE3F9CE5D90709F471C000F5E4
:103DC000C531FCE5DF0709F485C068F4C3319CE523
:103DD000D90709F475C008F095C00E945907809171
:103DE000E2028F77AFC0CC3FFCE5DF07A9F108F016
:103DF00054C0CB3FDC4509F0A7C08091E30240C02E
:103E0000C230EDE5DE0709F489C058F4C1158DE52F
:103E1000D80709F45AC008F069C08091E3028260B3
:103E20002FC0C236EDE5DE0709F47CC0C63AFDE5D9
:103E3000DF0709F481C0C330DD4509F085C080E0AB
:103E40006EC08091E20282607DC08091E20216C065
:103E50008091E202886076C08091E30282604FC068
:103E60008091E20280626EC08091E20280646AC04A
:103E70000E9459078091E202806864C0846062C039
:103E800081603DC08091E2028E7F5CC08091E20241
:103E90008D7F58C08091E20216C08091E30218C065
:103EA0008091E3028D7F2BC08091E2028F7E4AC019
:103EB0008091E2028F7D46C08091E2028F7B42C0FA
:103EC0008091E202877F8B7F3DC08091E3028D7FEE
:103ED0008E7F15C08091E20282FB222720F991E0BB
:103EE000922790FB82F990FB83F92CC08091E3022A
:103EF000982F909591708E7F892B90FB81F98093FC
:103F0000E30222C00E9459078091E20287FB222728
:103F100020F991E0922790FB87F914C081E00E947C
:103F2000390E12C08091E20284FB222720F991E031
:103F3000922790FB84F906C08091E202982F909519
:103F400090FB80F98093E2028091E2029091E3027B
:103F50000E94B30D0E94590780E001C081E0DF910B
:103F6000CF910895CF93DF9386319C4541F5EB01C6
:103F70000E94AC0C982F8A8120910201309103019C
:103F8000882379F09A7A81E009F480E08093B10285
:103F9000911102C069E201C065E3C9010E94A82134
:103FA0000AC08091B102811102C069E201C065E3DB
:103FB000C9010E94B3210E94EE0C80E001C081E0A3
:103FC000DF91CF9108950F931F93CF93DF93C42F69
:103FD000D22FFC0182818823C9F04093B4020E9451
:103FE0006C229093B3028093B20280E28C0F8830EF
:103FF00008F057C0C77081E001C0880FCA95EAF782
:10400000DF91CF911F910F910C94B6048091B4026F
:10401000481330C08091B2029091B3020E94842272
:10402000883C910538F510E21D0FCD17B9F080E2FC
:104030008C0F883040F4C77081E001C0880FCA95AA
:10404000EAF70E94BD04183028F581E09D2F977093
:1040500001C0880F9A95EAF70E94B604802F0E944B
:10406000AD041830F0F4D77081E001C0880FDA9504
:10407000EAF70AC080E28C0F883098F4C77081E0BC
:1040800001C0880FCA95EAF7DF91CF911F910F9178
:104090000C94BD04802FDF91CF911F910F910C9450
:1040A000AD04DF91CF911F910F9108950F939C0163
:1040B000CB01243F4CE5340731F188F4293DFCE580
:1040C0003F07D9F02A3D4CE5340779F1283D3C45BE
:1040D000A9F506E221EE41EE68ED7CE52BC0263F16
:1040E000FCE53F07E1F0A8F0273F3C4539F507E242
:1040F00025EE46EE67EF7CE51DC007E225EE45EEB6
:1041000069ED7CE517C006E221EE40EE64EF7CE548
:1041100011C007E225EE44EE65EF7CE50BC006E238
:1041200021EE42EE66EF7CE505C008E221E045EEB7
:104130006AED7CE50E94E31F80E008C0FC018281FB
:10414000882319F01092B40201C081E00F91089504
:104150009093C9018093C80108959093BA02809307
:10416000B9020895E091B902F091BA02309721F0B6
:104170000190F081E02D099480E00895E091B9026A
:10418000F091BA02309799F020912B01222359F037
:104190002091E20227FF07C0DC012C9111962C939D
:1041A000119726E02C930280F381E02D0994089565
:1041B000E091B902F091BA02309739F022E0DC01C7
:1041C0002C930480F581E02D099408952091B70285
:1041D0003091B8022817390771F09093B802809394
:1041E000B702E091B902F091BA02309721F006804F
:1041F000F781E02D099408952091B5023091B6021F
:104200002817390771F09093B6028093B502E091B8
:10421000B902F091BA02309721F00084F185E02DC7
:1042200009940895FC01329680912B01882331F086
:104230008091E20287FF02C09EE101C096E080E02B
:10424000915028F021912223D9F38F5FF9CF08955F
:10425000662351F120912B012223E9F02091E20203
:1042600027FF19C0462F4695469546954E31E0F4F6
:10427000677021E030E002C0220F331F6A95E2F739
:10428000FC01E40FF11D828190E02823392381E0B5
:10429000232B69F409C0FC0132960896219162171C
:1042A00029F0E817F907D1F780E0089581E0089533
:1042B0009C01FC0132969FEF80E04191461789F006
:1042C0009F3F19F4411101C0982F8F5F8630A9F7E5
:1042D0009F3F39F0F901E90FF11D97FDFA956283CF
:1042E000089508959C012A5F3F4FFC0142814613C7
:1042F00001C01282019682179307B9F70895262FFD
:104300002695269526952E3168F4FC01E20FF11DC5
:10431000677021E030E001C0220F6A95EAF78281E0
:10432000282B22830895262F2695269526952E3113
:1043300070F4FC01E20FF11D677021E030E001C074
:10434000220F6A95EAF72095828128232283089517
:1043500020912B01222329F02091E20227FD0C94C9
:104360007F210C94582120912B01222329F02091A8
:10437000E20227FD0C9493210C94722120912B01D1
:10438000FC013296222331F08091E20287FF02C0C5
:104390008EE101C086E0DF011D928A95E9F708955C
:1043A00008950C94D02183E08093BB020C94D1211A
:1043B000811102C081E001C082E08093BB020C94B5
:1043C000D1210C94D82181E08093BB020C94D1219F
:1043D0000C94E32108950C94EA210C94EB210C94A5
:1043E000EA210C94EA210C94EA21CF930E94F12156
:1043F0000E942E120E94EF21C0E08C2F0E945811C3
:10440000892B29F4CF5FC530C1F780E001C081E07E
:10441000CF91089508951F920F920FB60F92112415
:104420008F939F93AF93BF938091BC02811113C070
:1044300080913A0390913B03A0913C03B0913D03DE
:104440004196A11DB11D80933A0390933B03A09325
:104450003C03B0933D03BF91AF919F918F910F901B
:104460000FBE0F901F90189580914203843031F158
:104470000E947F031092BC0220E488E190E00FB616
:10448000F894A895809360000FBE2093600083B7D6
:10449000817F846083BF83B7816083BF7894889570
:1044A00083B78E7F83BF0FB6F894A8958091600084
:1044B000886180936000109260000FBE08950E9492
:1044C00059070C94860382E084BD93E095BD9AEF72
:1044D00097BD80936E0008952FB7F89480913A03AA
:1044E00090913B03A0913C03B0913D032FBF0895F1
:1044F0002FB7F89460913A0370913B0380913C038D
:1045000090913D032FBF08959C014FB7F89480917F
:104510003A0390913B03A0913C03B0913D034FBF00
:10452000821B930B089578941F920F920FB60F92EF
:1045300011248F939F93AF93BF9380913A039091EF
:104540003B03A0913C03B0913D030196A11DB11D19
:1045500080933A0390933B03A0933C03B0933D03B5
:10456000BF91AF919F918F910F900FBE0F901F90B1
:10457000189581E08093E00080E28093D80010924B
:10458000C9008FE19EE40197F1F700C0000087E0C9
:1045900090EBDC0180934B0390934C03A0934D036D
:1045A000B0934E039CE088E10FB6F894A8958093F1
:1045B00060000FBE90936000FFCF8091E0020895ED
:1045C000089522E02093E9002FEF3091E800215078
:1045D00035FD06C035ED3A95F1F700002111F5CF14
:1045E0002091E80025FF0BC040E050E066E070E05D
:1045F0000E9420258091E8008E778093E80008953E
:10460000CF93DF9320912B01222339F02091E202F6
:1046100027FF03C060E222E002C068E021E02093AF
:10462000E9002FEF3091E800215035FD06C035ED4F
:104630003A95F1F700002111F5CF2091E80025FF10
:104640001DC0EC0180912B01811105C040E050E0BC
:1046500068E070E003C070E040E050E0CE010E94EE
:1046600020258091E8008E778093E80080E2FE01AB
:10467000A0ECB2E001900D928A95E1F7DF91CF9125
:1046800008958093BD027093BF026093BE02809133
:104690004203843001F582E08093E9008FEF90912E
:1046A000E800815095FD06C095ED9A95F1F7000060
:1046B0008111F5CF8091E80085FF0DC040E050E00A
:1046C00063E070E08DEB92E00E9420258091E8008D
:1046D0008E778093E8000895BC0184E00C94412318
:1046E000BC0183E00C94412380914103811109C0F6
:1046F0000E94B1260E940E278091E2008460809380
:10470000E20008951092410308950C94E82160910D
:104710003E0381E0611101C080E00C94D3219091AF
:10472000420381E0943009F080E060913E030C94F4
:10473000D82142E061EC81E00E942A2642E261EC4D
:1047400082E00E942A269091420381E0943009F091
:1047500080E060913E030C94E1218091440383301A
:1047600009F461C030F4813071F0823009F49AC0EC
:1047700008958A3009F486C08B3009F46CC0893002
:1047800009F0A8C020C080914303813A09F0A2C07B
:104790008091E800877F8093E800809147039091A3
:1047A0004803892B21F460E280EC92E003C060E0D2
:1047B00080E090E070E00E946B258091E8008B77AC
:1047C0008093E800089580914303813209F082C00C
:1047D0008091470390914803029708F07BC0809135
:1047E000E800877F8093E8008091E80082FD05C0A3
:1047F000809142038111F8CF6DC02091F300809128
:10480000F20090E0922B029731F48091F100813018
:1048100011F0863021F48091F1008093E0028091C4
:10482000E8008B7753C080914303813A09F052C06E
:104830008091470390914803892B09F04BC08091E8
:10484000E800877F8093E8008091E80080FFFCCF3C
:1048500080912B0136C0809143038132D9F580913C
:10486000470390914803892BA9F58091E800877F41
:104870008093E8000E945F268091450380932B017E
:104880000C94590780914303813221F58091E8000F
:10489000877F8093E8000E945F2680914603809383
:1048A000E102089580914303813AA1F48091E800E8
:1048B000877F8093E8008091E80080FFFCCF8091A3
:1048C000E1028093F1008091E8008E778093E80008
:1048D0000C945F26089584B7877F84BF0FB6F89441
:1048E000A8958091600088618093600010926000BC
:1048F0000FBE90E080E80FB6F8948093610090932B
:1049000061000FBE0C94E3210E94B1260E940E2785
:10491000E2EEF0E080818460808378940C94A32997
:104920008FE191E00C94AD20809142038530A9F491
:1049300080914203853079F40E94342280914003B3
:104940008823B1F30E94F521882391F30E940A2560
:104950000E945907EDCF0C945F22089508950C949E
:10496000B124292F332723303105C9F060F42130D9
:10497000310581F02230310509F044C08BE390E02D
:104980002BEB33E043C021323105E1F02232310517
:1049900049F138C082E190E026EF33E037C0992733
:1049A0008130910549F028F0029761F5EFE8F3E0D6
:1049B00005C0E7EBF3E002C0EDEAF3E0849190E09C
:1049C0009F0124C06115710541F061307105D1F47A
:1049D00089E090E026EE33E019C089E090E02DEC0C
:1049E00033E014C06115710541F06130710551F477
:1049F00086EB90E028E034E009C080E490E02EEB04
:104A000034E004C080E090E020E030E0FA0131833F
:104A10002083089580E189BD82E189BD09B400FE4B
:104A2000FDCF8091D8008F7D8093D8008091E000E9
:104A300082608093E0008091E00081FDFCCF0895CA
:104A4000CF92DF92EF92FF920F931F93CF93DF935A
:104A5000EC018B017A010E947E26811133C0E114A2
:104A6000F10439F0F70180819181081B190BC80FFF
:104A7000D91FC12CD12C0115110519F18091E80025
:104A800085FD16C08091E8008E778093E800E114E0
:104A9000F10449F0F70180819181C80ED91ED182BD
:104AA000C08285E00FC00E947E26882321F30AC0C1
:104AB00089918093F10001501109FFEFCF1ADF0AAD
:104AC000DACF80E0DF91CF911F910F91FF90EF90AF
:104AD000DF90CF9008952091490330914A03261723
:104AE000370748F06115710539F42091E8002E77F9
:104AF0002093E80001C0B901FC0120E061157105B7
:104B000079F1809142038823F1F18530F1F18091B0
:104B1000E80083FD3CC08091E80082FD2EC08091BA
:104B2000E80080FFEBCF2091F3008091F20090E04D
:104B3000922B6115710551F08830910538F421915F
:104B40002093F100615071090196F3CF21E008979D
:104B500009F020E08091E8008E778093E800CECFC6
:104B60002111CFCF0AC080914203882361F08530A4
:104B700061F08091E80083FD0AC08091E80082FF27
:104B8000F2CF80E0089582E0089583E0089581E007
:104B900008952091490330914A032617370748F0BA
:104BA0006115710539F42091E8002E772093E80013
:104BB00001C0B901FC0120E06115710591F18091FE
:104BC0004203882309F440C0853009F43FC0809136
:104BD000E80083FD3DC08091E80082FD2FC08091F8
:104BE000E80080FFE9CF2091F3008091F20090E08F
:104BF000922B6115710559F08830910540F424918C
:104C00002093F1003196615071090196F2CF21E0B5
:104C1000089709F020E08091E8008E778093E80003
:104C2000CBCF2111CCCF0AC080914203882361F001
:104C3000853061F08091E80083FD0AC08091E80032
:104C400082FFF2CF80E0089582E0089583E0089526
:104C500081E00895982F973068F59093E9009817B0
:104C600039F07091EC002091ED005091F00003C0FC
:104C7000242F762F50E021FD02C09F5FECCF3091B2
:104C8000EB003E7F3093EB003091ED003D7F3093A1
:104C9000ED003091EB0031603093EB007093EC004D
:104CA0002093ED005093F0002091EE0027FDE5CF1A
:104CB00080E008958F708093E90081E008958091ED
:104CC000430387FF11C08091E80082FD05C08091F9
:104CD00042038111F8CF11C08091E8008B770BC09F
:104CE00080914203882349F08091E80080FFF8CF4B
:104CF0008091E8008E778093E80008952091E40089
:104D00003091E50095E64091EC00842F817040FFE2
:104D100023C08091E80080FD1DC08091420388235C
:104D200099F0853099F08091EB0085FD11C040919C
:104D3000E4005091E5002417350729F3915011F054
:104D40009A01E1CF84E0089582E0089583E0089518
:104D500081E0089580E008954091E80042FFDDCFB2
:104D600008950E941F270E942727E0EEF0E080812F
:104D700081608083E8EDF0E080818F77808319BCCB
:104D8000A7EDB0E08C918E7F8C9380818F7E8083A5
:104D90001092410308950F931F93CF93DF930E94C6
:104DA0001F270E942727C8EDD0E088818F7788834E
:104DB00088818068888388818F7D888319BC109260
:104DC000420310923E031092400310923F0300EE04
:104DD00010E0F80180818B7F8083888181608883E7
:104DE00042E060E080E00E942A26E1EEF0E080816F
:104DF0008E7F8083E2EEF0E080818160808380811D
:104E000088608083F80180818E7F808388818061C3
:104E10008883DF91CF911F910F910895E8EDF0E025
:104E200080818F7E8083E7EDF0E0808181608083E8
:104E300084E082BF81E0809341030C94CB26E8EDAF
:104E4000F0E080818E7F80831092E20008951092BE
:104E5000DA001092E10008951F920F920FB60F92A0
:104E600011242F933F934F935F936F937F938F936F
:104E70009F93AF93BF93EF93FF938091E10082FFE5
:104E80000BC08091E20082FF07C08091E1008B7F20
:104E90008093E1000E94A2298091DA0080FF1FC068
:104EA0008091D80080FF1BC08091DA008E7F8093B4
:104EB000DA008091D90080FF0DC080E189BD82E1D8
:104EC00089BD09B400FEFDCF81E0809342030E94BA
:104ED000742305C019BC109242030E948223809162
:104EE000E10080FF19C08091E20080FF15C0809131
:104EF000E2008E7F8093E2008091E20080618093E7
:104F0000E2008091D80080628093D80019BC85E0CF
:104F1000809342030E9487238091E10084FF30C088
:104F20008091E20084FF2CC080E189BD82E189BDCF
:104F300009B400FEFDCF8091D8008F7D8093D8000A
:104F40008091E1008F7E8093E1008091E2008F7E6E
:104F50008093E2008091E20081608093E200809182
:104F60003E03882311F084E007C08091E30087FDB1
:104F700002C081E001C083E0809342030E948F233E
:104F80008091E10083FF29C08091E20083FF25C06A
:104F90008091E100877F8093E10082E0809342036B
:104FA00010923E038091E1008E7F8093E10080911A
:104FB000E2008E7F8093E2008091E2008061809326
:104FC000E20042E060E080E00E942A268091F0004A
:104FD00088608093F0000E948523FF91EF91BF913C
:104FE000AF919F918F917F916F915F914F913F9181
:104FF0002F910F900FBE0F901F9018951F920F9238
:105000000FB60F9211242F933F934F935F936F939B
:105010007F938F939F93AF93BF93CF93DF93EF9340
:10502000FF93C091E900CF708091EC00D82FD17030
:1050300080FDD0E81092E9008091F000877F809396
:10504000F00078940E9442281092E9008091F000CC
:1050500088608093F000CD2BCF70C093E900FF9162
:10506000EF91DF91CF91BF91AF919F918F917F9100
:105070006F915F914F913F912F910F900FBE0F90C5
:105080001F9018951F93CF93DF93CDB7DEB7AA97E4
:105090000FB6F894DEBF0FBECDBFE3E4F3E080911E
:1050A000F100819323E0EB34F207C9F70E94AD23AE
:1050B0008091E80083FF2EC18091430390914403C7
:1050C000492F50E04A30510508F024C1FA01EE5949
:1050D000FF4F0C94262A803821F0823809F01AC13B
:1050E00008C080913F0390914003992389F082602A
:1050F0000FC0809147038F70873008F00BC18093F9
:10510000E9008091EB0085FB882780F91092E90087
:105110009091E800977F9093E8008093F1001092BF
:10512000F100D1C0282F2D7F09F0F4C0882319F099
:10513000823061F0EFC080914503813009F0EAC010
:10514000933009F080E0809340032EC080914503A6
:1051500081112AC0809147038F702FEF280F2630CE
:1051600008F0D8C08093E9002091EB0020FF1CC01C
:10517000933021F48091EB00806214C09091EB0099
:1051800090619093EB0021E030E0A90102C0440F50
:10519000551F8A95E2F74093EA001092EA00809149
:1051A000EB0088608093EB001092E9008091E800AA
:1051B000877F8093E8000E945F26ACC08111AAC05F
:1051C000109145031F778091E3008078812B8093B5
:1051D000E3008091E800877F8093E8000E945F26CB
:1051E0008091E80080FFFCCF8091E300806880938D
:1051F000E300111102C082E001C083E0809342030A
:1052000089C08058823008F085C080914503909114
:1052100046038C3D53E0950779F583E08A838AE263
:1052200089834FB7F894DE01139620E03EE051E207
:10523000E32FF0E050935700E49120FF03C0E29584
:10524000EF703F5FEF708E2F90E0EA3010F0C7965E
:1052500001C0C0968D939D932F5F243149F74FBFB6
:105260008091E800877F8093E8006AE270E0CE01D9
:1052700001960E946B2516C0609147037091480308
:10528000AE014F5F5F4F0E94AF24BC01892B09F430
:1052900041C09091E800977F9093E80089819A81BE
:1052A0000E94C9258091E8008B778093E80032C086
:1052B000803881F58091E800877F8093E8008091B5
:1052C0003E038093F1008091E8008E7772CF8111C8
:1052D00021C0809145039091460399270297D4F409
:1052E0008091E800877F8093E80080914503809358
:1052F0003E030E945F2680913E03811106C080918B
:10530000E30087FD02C081E001C084E08093420396
:105310000E9499238091E80083FF0AC08091E800F1
:10532000877F8093E8008091EB0080628093EB00A0
:10533000AA960FB6F894DEBF0FBECDBFDF91CF9116
:105340001F9108950895CF93809142038823A1F07F
:10535000C091E900CF709091EC00892F817090FD91
:1053600080E8C82B1092E9008091E80083FD0E943C
:105370004228CF70C093E900CF910895DB018F934D
:105380009F930E944A2ABF91AF91A29F800D911DC9
:10539000A39F900DB29F900D1124089587FB082EB6
:1053A000062687FD819567FD61950E945D2A0EF4B2
:1053B000919507FC81950895AA1BBB1B51E107C07D
:1053C000AA1FBB1FA617B70710F0A61BB70B881F95
:1053D000991F5A95A9F780959095BC01CD01089524
:1053E00097FB072E16F4009407D077FD09D00E9492
:1053F000DC2907FC05D03EF4909581959F4F0895D8
:10540000709561957F4F0895A1E21A2EAA1BBB1BD0
:10541000FD010DC0AA1FBB1FEE1FFF1FA217B30780
:10542000E407F50720F0A21BB30BE40BF50B661F96
:10543000771F881F991F1A9469F76095709580955A
:1054400090959B01AC01BD01CF010895EE0FFF1FA8
:105450000590F491E02D09940E94342A332312F42C
:105460008A1B9B0B0C94452AA29FB001B39FC001DD
:10547000A39F700D811D1124911DB29F700D811D80
:105480001124911D08950E94342AB7FF0895821BAC
:10549000930B08950E94342AA59F900DB49F900D00
:1054A000A49F800D911D11240895B7FF0C944A2AE2
:1054B0000E944A2A821B930B0895991B79E004C02D
:1054C000991F961708F0961B881F7A95C9F7809543
:1054D0000895FC014150504030F001900616D1F77C
:1054E0003197CF010895882799270895FB01DC01A2
:1054F00004C08D910190801921F441505040C8F7AB
:10550000881B990B0895F999FECF92BD81BDF89A39
:10551000992780B50895A6E1B0E044E050E00C94EE
:10552000BD2AA8E1B0E042E050E00C94BD2A262F4D
:10553000F999FECF92BD81BDF89A019700B4021689
:1055400039F01FBA20BD0FB6F894FA9AF99A0FBE37
:1055500008950396272F0E94982A0E94972A252FA4
:105560000E94982A242F0C94982A0196272F0E9493
:10557000982A0C94972ADC01CB01FC01F999FECF03
:1055800006C0F2BDE1BDF89A319600B40D924150CB
:0A5590005040B8F70895F894FFCFDB
:10559A00C8006002280850011E0A14010101020015
:1055AA001400141401191A1B1C1D1E1F202122DDB0
:1055BA00220023E12270236C23E02201E200E900A9
:1055CA00EA00B500B600B700CD008301CC008A011D
:1055DA0092019401210223022402250226022702B3
:1055EA002A02B300B4006F007000818283E200E9EE
:1055FA0000EA00B500B600B700CD008301CC008AEE
:10560A000192019401210223022402250226022783
:10561A00022A02B300B4006F007000818283F0F1A5
:10562A00C66766379431303534979633F4F59091DE
:10563A009293950001020202020606060909090967
:10564A0009090F0F0F0F0F0F151515181919191929
:08565A0019191919191923246B
:00000001FF
